:0200000480007A
:100000006F0000091300000013000000130000003F
:100010001300000013000000130000001300000094
:10002000732E2034631E0E00130FC0FFF32E103406
:10003000B3FEEE01938E4E0073901E346F00C0012C
:10004000B70E0080337FDE0163180F00F32E1034EB
:10005000938E4E0073901E34B70E0080938E3E0038
:100060006396CE01930E800073B04E34B70E0080BD
:10007000938E7E006394CE0173504030B70E0080A3
:10008000938EBE006394CE017350403073002030D5
:10009000130E100073000000130E20009302800066
:1000A00073A002309302800073904230930280006C
:1000B00073A042341300000013000000130000007E
:1000C00013000000130000001300000013000000E4
:1000D00013000000130000001300000013000000D4
:1000E00013000000130E300093020008739042309A
:1000F00013000000130000001300000013000000B4
:10010000130000001300000013000000130E400055
:10011000B7120000938202807390423013000000F7
:100120001300000013000000130000001300000083
:100130001300000013000000130E5000B70110F070
:10014000938101F403A2010083A241001302F23F54
:1001500023A4410023A65100130E600013020008DF
:1001600073104230130E700073005010130E800095
:100170009301100023A04100130E90002390410032
:10018000130EA00003A20100130EB00003920100A1
:10019000130EC000130ED00083200000130EE000E9
:1001A00073002020130EF000B70010F0938000F6CB
:1001B00003A10000130E000123A02000130E100164
:0401C0006780000054
:1001C4006780000013050000678000001000000035
:1001D40000000000017A5200017C01011B0D0200A5
:1001E4001000000018000000DCFFFFFF0800000002
:1001F40000000000100000002C000000C4FFFFFFFE
:080204000400000000000000EE
:0400000580000090E7
:00000001FF
